:020000040800F2
:1000000000040020E1010008CD0E0008D10E000818
:10001000250F0008D10E0008F90E0008E3010008C2
:10002000E3010008E3010008E3010008C526000819
:10003000E3010008E3010008E3010008E301000810
:10004000E3010008E3010008E3010008E301000800
:10005000E3010008E30100082538000851380008D2
:100060007D380008A9380008D5380008E3010008E9
:10007000E3010008E3010008E3010008E3010008D0
:10008000E3010008E3010008E3010008E3010008C0
:10009000E3010008E3010008E3010008013900085A
:1000A000E3010008E3010008E3010008E3010008A0
:1000B000E3010008E3010008E3010008E301000890
:1000C000E3010008E3010008E3010008E301000880
:1000D000E3010008E3010008B50F0008E301000890
:1000E00069390008E3010008E3010008E3010008A2
:1000F000E3010008E3010008E3010008E301000850
:10010000E3010008E30100083D360008E3010008B0
:10011000E3010008E3010008E3010008E30100082F
:10012000E3010008E3010008E3010008E30100081F
:10013000E3010008E3010008E3010008E30100080F
:10014000E3010008E3010008E3010008B12D000805
:10015000E3010008E3010008E3010008E3010008EF
:10016000E3010008E3010008E3010008E3010008DF
:10017000E3010008E3010008E3010008E3010008CF
:10018000E3010008E3010008E3010008E3010008BF
:10019000E3010008E3010008E3010008E3010008AF
:1001A000E3010008E3010008E3010008E30100089F
:1001B000E3010008E3010008E3010008E30100088F
:1001C000E3010008E3010008E3010008E30100087F
:1001D000E3010008E3010008E3010008E30100086F
:1001E00002E000F000F8FEE772B6394880F30888B4
:1001F000384880F3098838484EF60851CEF200019D
:10020000086040F20000CCF200004EF63471CEF2ED
:1002100000010860BFF34F8FBFF36F8F40F2000003
:10022000C0F2F0004EF68851CEF200010860BFF334
:100230004F8FBFF36F8F4FF00000E1EE100A4EF6C4
:100240003C71CEF200010860062080F31488BFF3F1
:100250006F8F02F075FA03F087F94FF055301F49A0
:100260001B4A91423CBF41F8040BFAE71C49194A6A
:1002700091423CBF41F8040BFAE71A491A4A1B4B5A
:100280009A423EBF51F8040B42F8040BF8E70020F5
:100290001749184A91423CBF41F8040BFAE702F0B3
:1002A00053FA03F0BDF9144C144DAC4203DA54F880
:1002B000041B8847F9E700F03FF8114C114DAC42A0
:1002C00003DA54F8041B8847F9E702F03BBA000050
:1002D000000400200024002000000008000000208E
:1002E00000040020C03D0008002400202824002035
:1002F0002824002090340020E0010008E0010008DC
:10030000E0010008E00100082DE9F04F2DED108A12
:10031000C1F80CD0C3689D46BDEC108ABDE8F08FD3
:10032000002383F311882846A047002001F056FEE1
:1003300001F006FE00DFFEE71B4B142270B51A70B9
:100340006FF03F0200245A720F225C709C70DC70C8
:100350001C715C719C71DC711C729A72DC7202F00F
:1003600083F9064602F0A8F9054650B90F4B9E42A4
:1003700017D001339E4241F2883412BF0546002453
:100380000125002002F07AF90DB100F0B5F800F077
:1003900045FD00F019FC204600F00CF900F0ACF827
:1003A000F9E70446EDE700BF28240020010007B06C
:1003B00008B500F087FBA0F120035842584108BD62
:1003C00007B5054B02211B88ADF8043001A800F0E9
:1003D000E5FB03B05DF804FB503A0008064991F8CC
:1003E000243033B100230822086A81F8243000F059
:1003F0000DBC0120704700BF482400202DE9F84FB4
:10040000234C94F824300546884617468BBB2E466D
:10041000DFF87C90002F38D094F824A0BAF1000FB8
:1004200005D12022FF214846266200F0E5FCCAF1F2
:100430000805BD4228BF3D465FFA85FBAD00414639
:100440002A4604EB8A0000F0ADFC94F82430A7EBB8
:100450000B079B445FFA8BFBBBF1080F2E44A844AB
:10046000FFB284F824B0D5D1FFF7B8FF0028D1D16E
:1004700008E0266A06EB8306B042C9D0FFF7AEFF5C
:100480000028C4D10020BDE8F88F0120BDE8F88F16
:100490004824002010B5202383F311881248C36834
:1004A0000BB101F021FE0023104A0F484FF47A717E
:1004B00001F0DEFD002383F311880D4C236813B196
:1004C0002368013B2360636813B16368013B636089
:1004D000084B1B7833B9636823B9022000F050FC45
:1004E0003223636010BD00BF34240020950400084F
:1004F000782500207024002010B5254B254953F89D
:10050000042F013200D110BD8B42F8D1224C234B75
:1005100022689A423AD9224B9B6803F1006303F5A3
:1005200080439A4232D2002000F068FB1D4B02202B
:10053000187000F017FC1C4B1A6C00221A64196E1C
:100540001A66196E596C5A64596E5A665A6E5A690F
:1005500042F080025A615A6922F080025A615A6957
:100560001A6942F000521A611A6922F000521A61A7
:100570001B6972B60D4A0E4B13601B68226820215E
:1005800081F311889D4683F30888104710BD00BF92
:10059000FC3F00081C40000804400008FF3F000822
:1005A00028240020702400200038024008ED00E0DC
:1005B000004000082DE9F04F99B0B34C0190202283
:1005C000FF2110A8A66800F017FCB04A1378A346D4
:1005D000A3B9AF480121C3601170202383F31188B0
:1005E000C3680BB101F080FD0023AA4AA8484FF46C
:1005F0007A7101F03DFD002383F31188019B13B153
:10060000A54B019A1A60A54AA349019F02920023B3
:1006100013704B6099461C461D469846012000F019
:10062000A1FB002F00F012829B4B1B68002B40F0B7
:100630000D8219B0BDE8F08F0220FFF7B9FE002847
:1006400040F0FB81019BB9F1000F08BF1F46944B9E
:100650001B88ADF82C3002210BA800F09FFADDE7D3
:100660004FF47A7000F02EFA031E0393EADB0220A7
:10067000FFF79EFE82460028E4D0039B581E042804
:1006800000F2DD81DFE800F0030E1114170018A856
:10069000052340F8343D042100F080FA54464FF021
:1006A000000856E004217848F6E704217D48F3E786
:1006B00004217D48F0E71C24204600F0A1FA043410
:1006C0000B9004210BA800F069FA2C2CF4D1E5E77B
:1006D000002DB7D0002CB5D00220FFF769FE0546EB
:1006E000002800F0AF8101206C4C00F087FA022056
:1006F000207000F037FB4FF000095FFA89FA50468E
:1007000000F08CFA074658B1504600F097FA09F10C
:1007100001090028F1D12C46A9460027634B97E731
:1007200001230220237000F011FB3E46DBF8083065
:100730009E4206D2304600F063FA0130EBD1043617
:10074000F4E7029B00261E70534BA9465E602C46C0
:10075000374600F059FB15B1002C18BF0027FFF7F2
:100760002FFE5BE7002D3FF46DAF002C3FF46AAF26
:10077000029B0220187000F0F5FA322000F0A2F976
:10078000B0F1000AC0F25E811AF0030540F05A8110
:10079000DBF8082006EB0A03934200F25381BAF516
:1007A000807F00F24F8155450DDA4FF47A7000F0EA
:1007B00089F90490049B002BC0F244813C4A049BBD
:1007C000AB540135EFE7C820FFF7F2FD05460028DE
:1007D00000F038811F2E11D8C6F12004544528BFDF
:1007E000544610AB26F0030022463149184400F06D
:1007F000D9FA2246FF212E4800F0FEFA4FEAAA0A53
:100800005FFA8AF22A493046FFF7F8FD04460028CD
:1008100000F01A8106EB8A0605469AE70220FFF7E8
:10082000C7FD00283FF40EAFFFF7D8FD00283FF4C6
:1008300009AF4FF0000A5346DBF8082092451CD25E
:10084000BAF11F0F12D8109A01320FD02AF003020A
:1008500018A90A4452F8202C0B92184604220BA91E
:1008600000F074FB0AF1040A0346E5E750460393DF
:1008700000F0C6F9039B0B90EFE718A8042140F89D
:100880004C3D00F08BF964E72824002074250020FB
:1008900034240020950400087825002070240020CE
:1008A000523A00082C24002030240020543A00083A
:1008B0007424002018A8002340F8343D642100F07F
:1008C00039F900287FF4BEAE0220FFF771FD002841
:1008D0003FF4B8AE0B9800F0C3F918AB43F8480DDD
:1008E00004211846CDE718A8002340F8343D6421C0
:1008F00000F020F900287FF4A5AE0220FFF758FD94
:1009000000283FF49FAE0B9800F0B8F918AB43F8FD
:10091000440DE5E70220FFF74BFD00283FF492AEBF
:1009200000F0B2F918AB43F8400DD9E70220FFF709
:100930003FFD00283FF486AE0BA9142000F0AAF971
:10094000824618A8042140F83CAD00F027F9514632
:100950000BA896E7322000F0B5F8B0F1000AFFF6D8
:1009600071AE1AF0030F7FF46DAEDBF808200AEBCE
:10097000080393423FF666AE0220FFF719FD0028F8
:100980003FF460AE2AF0030AC244D0453FF4E1AE22
:10099000404600F035F904210A900AA800F0FEF85C
:1009A00008F10408F1E74FF47A70FFF701FD002821
:1009B0003FF448AEFFF712FD00283FF4AFAE109BA6
:1009C00001330CD0082210A90020FFF717FD0028E2
:1009D0003FF4A4AE2022FF2110A800F00DFAFFF78B
:1009E000EFFC374801F000FB23E6002D3FF42AAE70
:1009F000002C3FF427AE18A8002340F8343D6421B2
:100A000000F098F8824600287FF41CAE0220FFF721
:100A1000CFFC00283FF416AE0390FFF7D1FC41F263
:100A2000883001F0E1FA0B9800F030FA00F0ECF9B0
:100A3000039B57461C461D46F0E5054689E64FF0E8
:100A40000008FFE52546FDE52C4667E6002000F09E
:100A500039F80490049B002BFFF6E3AD012000F071
:100A600075F9049B213B122B3FF6D8AD01A252F839
:100A700023F000BF3906000861060008D10600080F
:100A80001D0600081D0600081D0600086507000871
:100A9000550900081D080008B5080008E708000807
:100AA000150900081D0600082D0900081D0600088C
:100AB000A7090008530700081D060008EB090008F5
:100AC000A08601002DE9F34702AE00244FF47A75A9
:100AD00006F8014D144FDFF85880454397F9003070
:100AE0005A1C5FFA84F901D0A34212D158F82400AD
:100AF00003680122D3F820A031462B46D0470128B5
:100B000007D10A4B9DF8070083F8009002B0BDE8BA
:100B1000F0870134022CE1D14FF4FA7001F064FA4D
:100B20004FF0FF30F2E700BF00240020982500209E
:100B3000943A00082DE9F0474FF47A75144FDFF826
:100B4000588006464D43002497F900305A1C5FFA3E
:100B500084F901D0A34210D158F82400036804227C
:100B6000D3F820A031462B46D047042805D1094BA5
:100B700083F800900020BDE8F0870134022CE3D117
:100B80004FF4FA7001F030FA4FF0FF30BDE8F08713
:100B90000024002098250020943A000830B4074B28
:100BA0001A78074B53F822402368DD69054B0A4643
:100BB000AC460146204630BC604700BF9825002067
:100BC000943A0008A086010070B501F051FC094C70
:100BD000094E2070002530682378834208D901F03F
:100BE00041FC336805440133B5F5804F3360F2D3DF
:100BF00070BD00BF992500208025002001F0E6BCD3
:100C000000F1006000F580400068704700F100606E
:100C1000920000F5804001F071BC0000054B1A689D
:100C2000054B1B789B1A834202D9104401F01ABC71
:100C300000207047802500209925002038B5074DF9
:100C400004462868204401F015FC28B9286820448F
:100C5000BDE8384001F026BC38BD00BF802500202B
:100C600010F0030308D1B0F5007F05D800F1005063
:100C7000A0F508400068704700207047014BC0583D
:100C8000704700BF107AFF1F014B1868704700BF04
:100C9000002004E070B52A4B1C68C4F30B03240C3D
:100CA00063B140F21342934231D040F21942934271
:100CB0002FD040F2214293422DD10323214A0C250B
:100CC00005FB03235D6893F9082042F201039C426F
:100CD00024D0B4F5805F23D041F201039C4221D09F
:100CE00041F203039C421FD041F207039C4208BF1C
:100CF0003122441E0C44013D0B46A3421ED215F97D
:100D0000016F581C96B1034600F8016CF5E701230A
:100D1000D4E70223D2E73F220B4DD6E73322E3E7A5
:100D20004122E1E75A22E4E75922E2E72C258442F6
:100D30001D7001D9981C5A70401A70BD1846FBE707
:100D4000002004E0643A0008583A0008022803D161
:100D50000822034B9A6170470128FCD10422F8E76E
:100D600000100240022804D14FF40022034B9A6184
:100D700070470128FCD14FF48022F7E700100240B1
:100D8000022805D1064A536983F00803536170476E
:100D90000128FCD1024A536983F00403F6E700BF3F
:100DA0000010024010B50023934203D0CC5CC45421
:100DB0000133F9E710BD000030B5441E14F9010FEE
:100DC0000B4660B193F90050854201F1010106D153
:100DD0001AB993F90020801A30BD013AEEE7002AD3
:100DE000F7D1104630BD000002460346981A13F9A9
:100DF000011B0029FAD1704702440346934202D0F6
:100E000003F8011BFAE77047024B1A78024B1A707D
:100E1000704700BF982500200024002038B5154CED
:100E2000154D204600F028FC2946204600F050FCD5
:100E30002D6812486A6DD2F8043843F00203C2F8F4
:100E4000043801F0D1F80E49284600F04DFD6A6DD6
:100E50000C48D2F804380C4923F00203C2F80438D5
:100E6000A0424FF4E1330B6003D0BDE8384000F0FE
:100E700061BB38BDC42A0020743B000840420F000B
:100E80009C3B00081C2600208425002038B50B4B15
:100E90001A780B4B53F822400A4B9C4205460CD063
:100EA000094B002118461422FFF7A6FF05600146F2
:100EB0002046BDE8384000F03DBB38BD98250020F5
:100EC000943A0008C42A002084250020FEE7000090
:100ED00000B59BB0EFF3098168226846FFF762FF17
:100EE000EFF30583034B9A6B9A6A9A6A9A6A9A6A35
:100EF0009B6AFEE700ED00E000B59BB0EFF30981CF
:100F000068226846FFF74EFFEFF30583044B9A6BA8
:100F10009A6A9A6A9A6A9A6A9A6A9B6AFEE700BF14
:100F200000ED00E000B59BB0EFF309816822684650
:100F3000FFF738FFEFF30583034B5A6B9A6A9A6AFF
:100F40009A6A9A6A9B6AFEE700ED00E030B5084DA8
:100F50000A4491420BD011F8013B09245840013C4E
:100F6000F7D040F300032B4083EA5000F7E730BD91
:100F70002083B8ED002304491A465A50C818083394
:100F8000802B4260F9D170479C250020024AD3682B
:100F900043F0C003D360704700440040044B5A68DC
:100FA00010439A6858600AB1181D1047704700BF77
:100FB0001C2600202DE9F0413D4ED6F85C54EF6828
:100FC0002B68DA059CB20CD5202383F311884FF4EB
:100FD0000070FFF7E3FF6FF480732B60002383F34F
:100FE0001188202383F31188DFF8C48014F02F03C5
:100FF00031D183F31188380613D5210611D520236A
:1010000083F311882B4800F0F3F9002844DA082014
:10101000FFF7C4FF4FF67F733B40EB60002383F381
:1010200011887A060DD563060BD5202383F311882A
:10103000F26C336D9A4201D1336C7BBB002383F396
:101040001188D6F86424D3680BB110699847BDE8BD
:10105000F04101F047BB230712D014F0080F0CBF7A
:1010600000208020E10748BF40F02000A20748BFD1
:1010700040F04000630748BF40F48070FFF78EFFE8
:10108000A4066B6805D596F860144046194000F038
:101090005FFA2C68A4B2A9E76860BFE727F04007B1
:1010A0003F0410203F0CFFF779FFEF60C6E700BF59
:1010B0001C2600205426002010B5054C054A0021AE
:1010C000204600F015FA044BC4F85C3410BD00BF94
:1010D0001C2600208D0F00080044004038B5294C24
:1010E000037C002918BF0C46012B0546C0F8644458
:1010F00010D1254B98420DD1244B1A6C42F400328A
:101100001A641A6E42F400321A660B2126201B6EF6
:1011100000F046F81E4BD5F85C249A42236802D0B2
:101120001C498A422BD11C4901EB5301B1FBF3F35B
:10113000A188080442BF23F0070003F0070343EA35
:1011400040039360E38843F040039BB2136123891B
:1011500043F001039BB2536141F4045343F02C0369
:10116000D36001F4A05100231360B1F5806F1368C0
:1011700053680CBF7F23FF2385F8603438BD0749CF
:10118000D2E700BFBC3A00081C260020003802400D
:10119000001001400014014000BD010580DE800206
:1011A00000F1604300F01F02400903F561430901AB
:1011B0008000C9B200F1604083F8001300F561407F
:1011C00001239340C0F8803103607047F8B515469D
:1011D00082680669AA420B46816938BF8568761A1B
:1011E000B542044607D218462A46FFF7DBFDA3693D
:1011F0002B44A3610DE011D932461846FFF7D2FD0A
:10120000AF1B3A46E1683044FFF7CCFDE2683A4450
:10121000A261A3685B1BA3602846F8BD18462A4656
:10122000FFF7C0FDE368E4E783682DE9F041044679
:1012300093421546266938BF85684069361AB5421B
:101240000F4606D22A46FFF7ADFD63692B44636162
:101250000DE012D93246A5EB0608FFF7A3FD424682
:10126000B919E068FFF79EFDE26842446261A36835
:101270005B1BA3602846BDE8F0812A46FFF792FD7C
:10128000E368E4E710B50A440024C361029B0060F0
:1012900040608460C160816141610261036210BD90
:1012A00008B582694369934201D1826882B9826834
:1012B000013282605A1C42611970426903699A4284
:1012C00001D3C3684361002100F0AAFE002008BDDD
:1012D0004FF0FF3008BD000070B5202304460E46D5
:1012E00083F31188A568A5B1A368A269013BA36037
:1012F000531CA36115782269934224BFE368A3615C
:10130000E3690BB120469847002383F311882846F0
:1013100070BD3146204600F073FE0028E2DA85F306
:10132000118870BD2DE9F74F05460F4690469A4645
:10133000D0F81C90202686F311884FF0000B14463D
:1013400064B1224639462846FFF740FF034668B994
:101350005146284600F054FE0028F1D0002383F3C4
:101360001188A8EB040003B0BDE8F08FB9F1000FBD
:1013700003D001902846C847019B8BF31188E41ADB
:101380001F4486F31188DBE7C16081614161C3615D
:101390001144009B006040608260016103627047FD
:1013A000F8B504460E461746202383F31188A56836
:1013B000A5B1A368013BA36063695A1C62611E70FA
:1013C000236962699A4224BFE3686361E3690BB1F0
:1013D00020469847002080F31188F8BD3946204602
:1013E00000F00EFE0028E2DA85F31188F8BD000057
:1013F000836942699A4210B501D182687AB98268DC
:10140000013282605A1C82611C7803699A4201D3BE
:10141000C3688361002100F003FE204610BD4FF039
:10142000FF3010BD2DE9F74F05460F4690469A460E
:10143000D0F81C90202686F311884FF0000B14463C
:1014400064B1224639462846FFF7EEFE034668B9E6
:101450005146284600F0D4FD0028F1D0002383F344
:101460001188A8EB040003B0BDE8F08FB9F1000FBC
:1014700003D001902846C847019B8BF31188E41ADA
:101480001F4486F31188DBE702684368114301605B
:1014900003B11847704700001430FFF743BF000046
:1014A0004FF0FF331430FFF73DBF00003830FFF737
:1014B000B9BF00004FF0FF333830FFF7B3BF000073
:1014C0001430FFF709BF00004FF0FF311430FFF771
:1014D00003BF00003830FFF763BF00004FF0FF325A
:1014E0003830FFF75DBF000000207047FFF7E4BD14
:1014F00037B50F4B0360002343608360C360012353
:1015000004460374154600900B464FF4007200F138
:101510005C011430FFF7B6FE00942B464FF40072C6
:1015200004F5177104F13800FFF72EFF03B030BD4A
:10153000D03A000810B52023044683F31188FFF742
:10154000CDFD02232374002383F3118810BD000016
:1015500038B5C36904460D461BB904210844FFF79A
:1015600093FF294604F11400FFF79AFE002806DADB
:10157000201D4FF48061BDE83840FFF785BF38BDBE
:10158000026843681143016003B1184770470000C7
:1015900013B5446BD4F894341A681178042915D122
:1015A000217C022912D11979128901238B4013421F
:1015B0000CD101A904F14C0001F04AFED4F8944486
:1015C000019B21790246206800F0DAF902B010BDD3
:1015D000143001F0CDBD00004FF0FF33143001F0A6
:1015E000C7BD00004C3001F09FBE00004FF0FF333C
:1015F0004C3001F099BE0000143001F09BBD00009A
:101600004FF0FF31143001F095BD00004C3001F077
:101610006BBE00004FF0FF324C3001F065BE0000A1
:10162000D0F8942438B5136819780429054601D0F8
:10163000012038BD017C0229FAD112795C89012090
:1016400090400440F4D105F1140001F02DFD024654
:101650000028EDD0D5F894544FF480732868697948
:1016600000F07CF9204638BD406BFFF7D9BF000081
:1016700000207047704700007FB5124B03600023C5
:1016800043608360C360012502260F4B0574044646
:101690000290019300F18402294600964FF4807372
:1016A000143001F0DDFC094B0193029400964FF4D5
:1016B000807304F52372294604F14C0001F0A4FD67
:1016C00004B070BDF83A00086916000891150008CA
:1016D0000B68202282F311880A7903EB8202906161
:1016E0004A79093243F822008A7912B103EB820366
:1016F000986102230374C0F89414002383F31188C3
:101700007047000038B5037F044613B190F8543099
:10171000ABB9201D01250221FFF732FF04F11400AF
:1017200025776FF0010100F087FC84F8545004F134
:101730004C006FF00101BDE8384000F07DBC38BDC1
:1017400010B5012104460430FFF71AFF0023237768
:1017500084F8543010BD000038B50446002514301C
:1017600001F096FC04F14C00257701F065FD201D89
:1017700084F854500121FFF703FF2046BDE83840AC
:10178000FFF74EBF90F8443003F06003202B19D1CF
:1017900090F84520212A0AD0222A4FF000030ED0CB
:1017A000202A0FD1084A82630722C26304E0064B55
:1017B00083630723C36300230364012070478363AB
:1017C000C363F9E70020704701240020D0F8943467
:1017D00037B51A681178042904461AD1017C022908
:1017E00017D11979128901238B40134211D100F1CD
:1017F0004C05284601F0E0FD58B101A9284601F04A
:1018000027FDD4F89444019B21790246206800F01A
:10181000B7F803B030BD000000EB8103F7B59C6959
:1018200005460E46F4B1202383F3118805EB8607A5
:10183000201D0821FFF7A4FEFB685B691B684C3480
:1018400013B1204601F012FD01A9204601F000FD70
:10185000024648B1019B3146284600F091F800232A
:1018600083F3118803B0F0BDFB685A691268002A3F
:10187000F5D01B8A013B1340F1D105F14402EAE7A0
:10188000093138B550F82140DCB1202383F31188A9
:10189000D4F894241368527903EB8203DB689B69C4
:1018A0005D6845B104216018FFF76AFE294604F11E
:1018B000140001F003FC2046FFF7B2FE002383F37F
:1018C000118838BD7047000000F0C4BF01230370C9
:1018D00000234360C36183620362C36243620363A4
:1018E000038143817047000038B50446202383F309
:1018F000118800254160C56005614561856100F082
:10190000B9FF0223237085F3118838BD70B500EB51
:10191000810305465069DA600E46144618B110225C
:101920000021FFF769FAA06918B110220021FFF722
:1019300063FA31462846BDE8704001F065B8000002
:10194000028902F001020281428902F00102428111
:10195000002202614261826101F0EAB8F0B400EB5A
:1019600081044789E4680125A4698D403D43458190
:1019700023600023A2606360F0BC01F005B90000A1
:10198000F0B400EB81040789E468012564698D40A7
:101990003D43058123600023A2606360F0BC01F039
:1019A0007FB9000070B50223002504460370A0F83B
:1019B0004C5080F84E5080F84F5005814581C560ED
:1019C00005614561856180F8345000F0B9FF6368B6
:1019D0001B6823B129462046BDE87040184770BDFA
:1019E000436802781B6880F85020052202700BB112
:1019F0000421184770470000436890F850201B6886
:101A000002700BB1052118477047000090F8343080
:101A100070B5044613B1002380F8343004F1440259
:101A2000204601F0A7F863689B6863BB94F84450B4
:101A300015F0600615D194F8453005F07F0545EAAC
:101A4000032540F202339D4200F00E815BD8022D47
:101A500000F0DC803FD8002D00F08780012D00F0E1
:101A6000CF800021204601F0DDFA0021204601F060
:101A7000CFFA63681B6813B10621204698470623F6
:101A800084F8343070BD204698470028CED094F8B2
:101A90004B2094F84A3043EA0223E26B934238BF6A
:101AA000E36394F94430E56B002B4FF0200380F2A0
:101AB000FD80002D00F0EC80092284F8342083F3AF
:101AC00011880021E36BA26B2046FFF759FF00232A
:101AD00083F3118870BDB5F5817F00F0B180B5F555
:101AE000407F49D0B5F5807FBBD194F84630012BBB
:101AF000B7D1B4F84C3023F00203A4F84C30A663FD
:101B0000E6632664C3E740F201639D421ED8B5F543
:101B1000C06F3BD2B5F5A06FA3D1B4F84430B3F594
:101B2000A06F0ED194F8463084F84E30204600F075
:101B30005FFF63681B6813B10121204698470323A8
:101B400023700023A363E3632364A0E7B5F5106F5C
:101B500032D040F602439D4252D0B5F5006F80D19D
:101B600004F14F03A363012324E004F14C03A363B6
:101B70000223E36325648AE794F84630012B7FF45F
:101B800070AFB4F84C3043F00203B6E794F8492044
:101B9000616894F848304D6894F8471043EA02238E
:101BA000204694F84620A84700283FF45AAF4368DF
:101BB000A3630368E363A4E72378042B10D12023F5
:101BC00083F311882046FFF7BBFE86F31188636814
:101BD00084F84F601B68032121700BB120469847A1
:101BE00094F84630002BACD084F84F300423237097
:101BF00063681B68002BA4D0022120469847A0E709
:101C0000374BA3630223E36300239DE794F8481056
:101C100011F0800F204601F00F010ED000F09CFF64
:101C2000012806D002287FF41CAF2E4BA363E0638B
:101C300067E72D4BA363E56363E700F07FFFEFE702
:101C400094F84630002B7FF40CAF94F8483013F032
:101C50000F013FF476AF1A06204602D501F0F6F9DF
:101C60006FE701F0E9F96CE794F84630002B7FF458
:101C7000F8AE94F8483013F00F013FF462AF1B0642
:101C8000204602D501F0CEF95BE701F0C1F958E733
:101C9000142284F8342083F311882B462A462946DF
:101CA0002046FFF75BFE85F3118870BD5DB11522FC
:101CB00084F8342083F311880021E36BA26B204663
:101CC000FFF74CFE03E70B2284F8342083F31188DE
:101CD0002B462A4629462046FFF752FEE3E700BF7F
:101CE000283B0008203B0008243B000838B590F84A
:101CF00034300446152B29D8DFE803F03E28282885
:101D000028283E28280B2939282828282828282848
:101D10003E3E90F84B1090F84A20C36B42EA0122F5
:101D20009A4214D9C268128AB3FBF2F502FB153548
:101D30006DB9202383F311882B462A462946FFF7E5
:101D40001FFE85F311880A2384F8343038BD14232C
:101D500084F83430202383F3118800231A4619466F
:101D60002046FFF7FBFD002383F3118838BD036C89
:101D700003B198470023E7E7002101F053F9002160
:101D8000204601F045F963681B6813B1062120461F
:101D900098470623D8E7000090F83420152A38B574
:101DA000044622D80123934040F6416213421DD1DC
:101DB00013F480150FD19B0217D50B2380F8343014
:101DC000202383F311882B462A462946FFF7D8FDA6
:101DD00085F3118838BDC3689B695B682BB9036CB8
:101DE00003B19847002384F8343038BD002101F056
:101DF00019F90021204601F00BF963681B6813B143
:101E00000621204698470623EDE70000024B0022FA
:101E10001B605B609A607047842A00200023037473
:101E20008268054B1B6899689142FBD25A6803602F
:101E30004260106058607047842A002008B5202353
:101E400083F31188037C032B05D0042B0DD02BB911
:101E500083F3118808BD436900221A604FF0FF33F5
:101E60004361FFF7DBFF0023F2E790E80C001A6004
:101E700002685360F2E70000002303748268054B98
:101E80001B6899689142FBD85A68036042601060F1
:101E900058607047842A0020054B19690874186837
:101EA00002681A605360186101230374FEF72CBAAC
:101EB000842A002030B54B1C87B005460A4C10D050
:101EC00023690A4A01A800F0D3F82846FFF7E4FF87
:101ED000049B13B101A800F007F92369586907B002
:101EE00030BDFFF7D9FFF8E7842A00203D1E000827
:101EF00038B50C4D41612B6981689A68914204465E
:101F000003D8BDE83840FFF789BF1846FFF786FFC2
:101F100001232C61014623742046BDE83840FEF7BA
:101F2000F3B900BF842A0020044B1A681B6990682B
:101F30009B68984294BF002001207047842A0020AB
:101F400010B5084C236820691A6822605460012289
:101F500023611A74FFF790FF01462069BDE8104025
:101F6000FEF7D2B9842A0020826002220274002285
:101F7000427470478368A3F17C0243F80C2C026919
:101F800043F83C2C426943F8382C074A43F81C2C90
:101F9000C26843F8102C022203F8082C002203F830
:101FA000072CA3F1180070472103000810B5202367
:101FB00083F31188FFF7DEFF00210446FFF798FF47
:101FC000002383F31188204610BD0000024B1B69DB
:101FD00058610F20FFF760BF842A0020202383F37D
:101FE0001188FFF7F3BF000008B50146202383F3F3
:101FF00011880820FFF75EFF002383F3118808BDD6
:1020000049B1064B42681B6918605A60136043600F
:102010000420FFF74FBF4FF0FF307047842A0020A5
:102020000368984206D01A680260506059611846E9
:10203000FFF7F4BE7047000038B504460D4620682F
:10204000844200D138BD036823605C604561FFF7BE
:10205000E5FEF4E7054B03F114025A619A614FF073
:10206000FF32DA6100221A62704700BF842A002022
:10207000F8B503611A4BC2605C6A1A4B1A46022912
:1020800052F8145F38BF0221954206461F460AD116
:10209000586198611C620560456081600819BDE85F
:1020A000F84001F0ABB9186AAB68241A0C1902D3D6
:1020B000E41A2D6804E09C4202D2204401F0AEF9FB
:1020C000AB689C42F4D86B68736035601E606E60CC
:1020D000B460A9684FF0FF33091BA960FB61F8BD2C
:1020E000000C0040842A002010B41A4C234653F8F8
:1020F000141F814210D0416802680A600268516072
:102100009A424FF00001C16003D0936881680B448C
:1021100093605DF8044B70470A68626100209A4240
:102120005360C86003D15DF8044B01F071B9936846
:10213000886803449360084A206A526A121A9342DC
:10214000E7D9991A012998BF931C18445DF8044BEC
:1021500001F064B9842A0020000C00400020704780
:10216000FEE70000704700004FF0FF3070470000AE
:10217000022906D0032906D00129064818BF0020ED
:10218000704705487047032A9ABF044800EBC20015
:1021900000207047F83B0008AC3B000808240020F2
:1021A00070B59AB001AD064608462946144600F0BF
:1021B00095F82846FEF718FEC0B2431C5B0086E87F
:1021C0001800237003236370002302341946DAB227
:1021D000904204F1020401D81AB070BDEA5C04F820
:1021E000022C04F8011C0133F1E7000008B520239C
:1021F00083F311880348FFF7E9FA002383F311887A
:1022000008BD00BFC42A002010B50446052916D811
:10221000DFE801F016150316161D202383F311883D
:102220000E4A0121FFF772FB20460D4A0221FFF7FB
:102230006DFB0C48FFF790FA002383F3118810BD63
:10224000202383F311880748FFF75CFAF4E7202383
:1022500083F311880348FFF773FAEDE72C3B00087E
:10226000503B0008C42A002038B50C4D0C4C0D49D9
:102270002A4604F10800FFF793FF05F1CA0204F1B2
:1022800010000949FFF78CFF05F5CA7204F1180028
:102290000649BDE83840FFF783BF00BF8C2F002000
:1022A000082400207C3B0008863B0008913B000886
:1022B00070B5044608460D46FEF796FDC6B22046A8
:1022C000013403780BB9184670BD32462946FEF733
:1022D00073FD0028F3D1012070BD00002DE9F84FF7
:1022E00004460D46FEF780FD2849C6B22046FFF79A
:1022F000DFFF08B1033EF6B225492046FFF7D8FFBD
:1023000008B11036F6B2632E0DD8DFF88080DFF802
:102310008090204FDFF884A0DFF884B0267846B99B
:102320002E70BDE8F88F21462846BDE8F84F01F031
:1023300087BB252E26D1072241462046FEF73CFDCD
:1023400028B9DBF8003045F8043B0734E6E70822FB
:1023500049462046FEF730FDA0B90F4BAA1C13F8E2
:10236000011F09095345C95D02F8021C197801F0E3
:102370000F0102F10202C95D02F8031CEFD118350A
:102380000834CBE72E7001340135C7E7183C00084C
:10239000913B0008253C00080F7AFF1F1B7AFF1FA6
:1023A000203C0008BFF34F8F024AD368DB03FCD404
:1023B000704700BF003C024008B5094B1B7873B959
:1023C000FFF7F0FF074B1A69002ABFBF064A5A60A1
:1023D00002F188325A601A6822F480621A6008BDDD
:1023E000EA310020003C02402301674508B50B4B51
:1023F0001B7893B9FFF7D6FF094B1A6942F00042E8
:102400001A611A6842F480521A601A6822F48052E3
:102410001A601A6842F480621A6008BDEA3100202E
:10242000003C02400B2870B513D80B4A0B4C1378B4
:1024300063B90B4E4FF0006144F8231056F8235057
:1024400001330C2B2944F7D10123137054F82000D9
:1024500070BD002070BD00BF1C320020EC31002098
:10246000383C0008014B53F820007047383C000806
:102470000C2070470B2810B5044601D9002010BD70
:10248000FFF7D0FF064B53F824301844C21A0BB99B
:10249000012010BD12680132F0D1043BF6E700BF05
:1024A000383C00080B2810B5044621D8FFF77AFF06
:1024B000FFF782FF0F4AF323D360C300DBB243F47C
:1024C000007343F002031361136943F48033136113
:1024D000FFF768FFFFF7A6FF074B53F8241000F043
:1024E000DDF8FFF783FF2046BDE81040FFF7C2BFCD
:1024F000002010BD003C0240383C00082DE9F843A4
:1025000012F00103154640D18218B2F1016F3CD29E
:102510002C4B1B6813F0010337D02B4CFFF74CFFFB
:10252000F323E360FFF73EFF40F20127032D01D9BB
:10253000830713D0244C0F46401A40F20118EB1BBE
:102540000B44012B00EB0706236924D823F0010379
:102550002361FFF74BFF0120BDE8F883236923F4D3
:102560004073236123693B43236151F8046B066088
:10257000BFF34F8FFFF716FF03689E4208D0236911
:1025800023F001032361FFF731FF0020BDE8F8834A
:10259000043D0430CAE723F440732361236943EA0E
:1025A00008032361B94637F8023B3380BFF34F8FEE
:1025B000FFF7F8FE3688B9F80030B6B2B342BED0A5
:1025C000DDE700BF00380240003C0240084908B582
:1025D0000B7828B153B9FFF7EFFE01230B7008BD4C
:1025E00023B1BDE808400870FFF700BF08BD00BF79
:1025F000EA31002010B50244064B0439D2B29042B1
:1026000000D110BD441C00B253F8200041F8040F63
:10261000E0B2F4E750280040104B30B51C6F2404A2
:1026200007D41C6F44F400741C671C6F44F400440E
:102630001C670B4C236843F4807323600244094BEE
:102640000439D2B2904200D130BD441C00B251F8DE
:10265000045F43F82050E0B2F4E700BF00380240C6
:10266000007000405028004007B5012201A9002059
:10267000FFF7C0FF019803B05DF804FB13B50446F3
:10268000FFF7F2FFA04206D002A9012241F8044D53
:102690000020FFF7C1FF02B010BD0000704700002E
:1026A000034B1B689B0042BF024B01221A7070470C
:1026B000743802401D320020014B1878704700BF6B
:1026C0001D320020064A536823F001035360EFF3E4
:1026D0000983683383F30988002383F311887047E3
:1026E00030EF00E010B5202383F31188104B5B68B6
:1026F00013F4006318D0F1EE103AEFF309844FF0B1
:10270000807344F84C3C0B4BDB6844F8083CA4F164
:10271000680383F30988FFF707FC18B1064B44F8F8
:10272000503C10BD054BFAE783F3118810BD00BF84
:1027300000ED00E030EF00E0310300083403000852
:1027400070470000FEE70000084A094B09498B4228
:1027500004D3094A0021934205D3704752F8040F6D
:1027600043F8040BF3E743F8041BF4E7E43D0008E7
:10277000903400209034002090340020836D30B5D8
:1027800000229D68446D11464FF0FF3004EB421368
:1027900001329542C3F80019C3F81019C3F80809AB
:1027A000C3F8001BC3F8101BC3F8080BEED24FF0A0
:1027B0000113C4F81C3830BD890141F020010161CA
:1027C00003699B06FCD4122000F0B4BE204B03EB3F
:1027D00080022DE9F047D2F80CE05D6DDEF81420A0
:1027E000461CD2F800C005EB063605EB40185168D0
:1027F00061450BD3D5F83428012303FA00F022EA0F
:102800000000C5F834081846BDE8F087BEF810404F
:10281000ACEB0103A34228BF2346D8F81849A4B261
:10282000B3EB840F10D894681F46A4F1040959F83B
:1028300004AFC6F800A0042F01D9043FF7E71C44F9
:102840000B4494605360D2E70020BDE8F08700BFDE
:102850002032002010B5054C2046FFF737F84FF026
:10286000A0436365024BA36510BD00BF203200206A
:102870008C3C00080378012B70B5054650D12A4BDB
:10288000446D98421BD1294B5A6B42F080025A6327
:102890005A6D42F080025A655A6D5A6942F08002C0
:1028A0005A615A6922F080025A610E2143205B6905
:1028B000FEF776FC1E4BE3601E4BC4F80038002385
:1028C000C4F8003EC02323606E6D4FF40413A3636D
:1028D0003369002BFCDA012333610C2000F02AFE5F
:1028E0003369DB07FCD4122000F024FE3369002B8F
:1028F000FCDA0026A6602846FFF740FF6B68C4F8A4
:102900001068DB68C4F81468C4F81C684BB90A4B3B
:10291000A3614FF0FF336361A36843F00103A36039
:1029200070BD064BF4E700BF2032002000380240A3
:102930004014004003002002003C30C0083C30C07E
:10294000F8B5446D054600212046FFF735FFA96D17
:1029500000234FF001128F68C4F834384FF000663E
:10296000C4F81C284FF0FF3004EB431201339F42A0
:10297000C2F80069C2F8006BC2F80809C2F8080B77
:10298000F2D20B686A6DEB656362102313611669FE
:1029900016F01006FBD1122000F0CCFDD4F8003860
:1029A00023F4FE63C4F80038A36943F4402343F0E2
:1029B0001003A3610923C4F81038C4F814380A4B73
:1029C000EB604FF0C043C4F8103B084BC4F8003B29
:1029D000C4F81069C4F80039EB6D03F1100243F438
:1029E0008013EA65A362F8BD683C000840800010CF
:1029F000426D90F84E10D2F8003823F4FE6343EA9B
:102A00000113C2F8003870472DE9F0410EB200EB17
:102A100086080D46D8F80C100F6807F00303022B48
:102A200050D0032B50D03D4A3D4F012B18BF1746C5
:102A3000446D4FEA451E04EB0E030022C3F8102B31
:102A40008A6905F1100C002A40D04A8A05F1580322
:102A50005B013A43E2500123D4F81C2803FA0CF33B
:102A60001343A6444A69C4F81C380023CEF8103931
:102A700005F13F03002A39D00A8A898B920801297F
:102A800088BF4A43C16D04EB8303561841EA0242F2
:102A9000C66529465A602046FFF78EFED8F80C30EE
:102AA0001B8A43EA85531F4305F148035B01E75046
:102AB0000123D4F81C2803FA05F51543C4F81C5863
:102AC000BDE8F081174FB3E7174FB1E704EB4613AA
:102AD000D3F8002B22F40042C3F8002BD4F81C28B2
:102AE000012303FA0CF322EA0303BAE704EB83039E
:102AF0000E4A5A6004EB461629462046FFF75CFE54
:102B0000D6F8003923F40043C6F80039D4F81C384D
:102B1000012202FA05F523EA0505CFE7008000103F
:102B2000008004100080081000800C1000040002D7
:102B3000826D1268C265FFF721BE00005831436DF7
:102B400049015B5813F4004004D013F4001F14BF74
:102B500001200220704700004831436D49015B5855
:102B600013F4004004D013F4001F14BF012002200E
:102B70007047000000EB8101CB68196A0B68136095
:102B80004B6853607047000000EB810330B5DD688F
:102B9000AA691368D36019B9402B84BF402313601E
:102BA0006B8A1468426D1C44013CB4FBF3F463432C
:102BB000033323F0030302EB411043EAC44343F021
:102BC000C043C0F8103B2B6803F00303012B09B28C
:102BD0000ED1D2F8083802EB411013F4807FD0F800
:102BE000003B14BF43F0805343F00053C0F8003B58
:102BF00002EB4112D2F8003B43F00443C2F8003B21
:102C000030BD00002DE9F041244D6E6D06EB401300
:102C10000446D3F8087BC3F8087B38070AD5D6F8F2
:102C20001438190706D505EB84032146DB682846CE
:102C30005B689847FA072FD5D6F81438DB072BD5F1
:102C400005EB8403D968CCB98B69488A5E68B6FB0A
:102C5000F0F200FB12628AB91868DA6890420DD26D
:102C6000121A83E81400202383F311880B482146AD
:102C7000FFF78AFF84F31188BDE8F081012303FA8E
:102C800004F26B8923EA02036B81CB6823B12146EE
:102C90000248BDE8F0411847BDE8F081203200202D
:102CA00000EB810370B5DD68436D6C692668E660F2
:102CB0004A0156BB1A444FF40020C2F810092A6892
:102CC00002F00302012A0AB20ED1D3F8080803EB7E
:102CD000421410F4807FD4F8000914BF40F08050F3
:102CE00040F00050C4F8000903EB4212D2F800098A
:102CF00040F00440C2F80009D3F83408012202FA77
:102D000001F10143C3F8341870BD19B9402E84BFD6
:102D10004020206020682E8A841940F00050013C39
:102D20001A44B4FBF6F440EAC440C6E7F8B50446DA
:102D30001E48456D05EB4413D3F80869C3F80869CC
:102D4000F10717D5D5F81038DA0713D500EB84034F
:102D5000D9684B691F68DA68974218D2D21B0027DE
:102D60001A605F60202383F311882146FFF798FFE4
:102D700087F31188330617D5D5F834280123A340EB
:102D8000134211D02046BDE8F840FFF71FBD0123D4
:102D900003FA04F2038923EA020303818B68002B00
:102DA000E8D021469847E5E7F8BD00BF2032002073
:102DB00096482DE9F84F456D6E69AB691E4016F4D3
:102DC000805F6E61044605D0FEF7ECFDBDE8F84F6C
:102DD000FFF788BC002E12DAD5F8003E8B489B071F
:102DE0001EBFD5F8003E23F00303C5F8003ED5F81A
:102DF000043823F00103C5F80438FEF7FDFD37055C
:102E000002D58248FEF7ECFDB0040CD5D5F80838A1
:102E100013F0060FEB6823F470530CBF43F4105308
:102E200043F4A053EB60310704D56368DB680BB152
:102E300076489847F2025AD4B3020CD5D4F854809D
:102E4000DFF8C8A100274FF00109A36D9B68F9B214
:102E50008B4280F08780F70619D5616D0A6AC2F34C
:102E60000A1702F00F0302F4F012B2F5802F00F0FF
:102E7000A180B2F5402F0AD104EB830301F5805104
:102E8000DB68186A00231A469F4240F087803003AF
:102E9000D5F8184813D5E10302D50020FFF7B2FE9C
:102EA000A20302D50120FFF7ADFE630302D5022085
:102EB000FFF7A8FE270302D50320FFF7A3FE750343
:102EC00084D5E00702D50020FFF730FFA10702D527
:102ED0000120FFF72BFF620702D50220FFF726FF34
:102EE00023077FF573AF0320FFF720FF6EE7D4F8C9
:102EF0005480DFF818A100274FF00109A36D9B68EB
:102F00005FFA87FB5B4597D308EB4B13D3F8002997
:102F100002F44022B2F5802F22D1D3F80029002AF2
:102F20001EDAD3F8002942F09042C3F80029D3F802
:102F30000029002AFBDB5946606DFFF73DFC228922
:102F400009FA0BF322EA0303238104EB8B03DB680A
:102F50009B6813B15946504698475846FFF736FCD0
:102F60000137CBE708EB4112D2F8003B03F44023D2
:102F7000B3F5802F10D1D2F8003B002B0CDA628918
:102F800009FA01F322EA0303638104EB8103DB689E
:102F9000DB680BB150469847013756E79C0708BFDE
:102FA0000A68072B98BF027003F101039CBF120A45
:102FB000013069E7023304EB830201F58051526866
:102FC00090690268D0F808C04068A2EB000E0022A9
:102FD000104697420AD104EB830463689B699A68A0
:102FE0003A449A605A6817445F6050E712F0030F42
:102FF00008BF0868964588BF8CF8000002F10102FE
:1030000084BF000A0CF1010CE3E700BF203200206E
:10301000436D03EB4111D1F8003B43F40013C1F8B9
:10302000003B7047436D03EB4111D1F8003943F485
:103030000013C1F800397047436D03EB4111D1F81B
:10304000003B23F40013C1F8003B7047436D03EBD2
:103050004111D1F8003923F40013C1F80039704749
:1030600030B5039C0172043304FB0325C361049B48
:1030700003630021059B00604060C1604261026102
:103080008561046242628162C162436330BD0000B7
:103090000022416A41610161C2608262C2626FF0D6
:1030A0000101FEF7C9BF000003694269934203D1E1
:1030B000C2680AB100207047181D70470369196083
:1030C000C2680132C260C2691344826903619342DB
:1030D00024BF436A03610021FEF7A2BF38B504464E
:1030E0000D46E3683BB16269131D1268A362134485
:1030F000E362002038BD237A33B929462046FEF723
:103100007FFF0028EDDA38BD6FF00100FBE700001B
:10311000C368C269013BC360436913448269436168
:10312000934224BF436A436100238362036B03B16C
:103130001847704770B52023044683F31188866AC8
:103140003EB9FFF7CBFF054618B186F31188284634
:1031500070BDA36AE26A13F8015BA362934202D3D3
:103160002046FFF7D5FF002383F31188EFE7000027
:103170002DE9F84F04460E4690469946202787F3DE
:1031800011880025AA46D4F828B0BBF1000F09D158
:1031900049462046FFF7A2FF20B18BF3118828464D
:1031A000BDE8F88FA16AE36AA8EB050B5B1A9B45A3
:1031B00028BF9B46BBF1400F1BD9334601F14002AB
:1031C00051F8040B43F8040B9142F9D1A36A403340
:1031D0004036A3624035A26AE36A9A4202D320468F
:1031E000FFF796FF8AF311884545D8D287F31188F7
:1031F000C9E730465A46FDF7D5FDA36A5B445E44F5
:10320000A3625D44E7E7000010B5029C017204333D
:1032100003FB0421C36100238362C362039B036336
:10322000049B00604060C46042610261816104628D
:103230004262436310BD0000026AC260426A42619A
:10324000026100228262C2626FF00101FEF7F4BEE9
:10325000436902699A4203D1C2680AB100207047EB
:10326000184650F8043B0B6070470000C368C26901
:103270000133C3604369134482694361934224BFAD
:10328000436A43610021FEF7CBBE000038B5044617
:103290000D46E3683BB123691A1DA262E26913443B
:1032A000E362002038BD237A33B929462046FEF771
:1032B000A7FE0028EDDA38BD6FF00100FBE7000043
:1032C00003691960C268013AC260C2691344826925
:1032D0000361934224BF436A036100238362036B4B
:1032E00003B118477047000070B5202304460E460E
:1032F00083F31188856A35B91146FFF7C7FF10B10E
:1033000085F3118870BDA36A1E70A36AE26A013357
:103310009342A36204D3E16920460439FFF7D0FF4A
:10332000002080F3118870BD2DE9F84F04460D464A
:1033300091469A464FF0200888F311880026B3463C
:10334000A76A4FB951462046FFF7A0FF20B187F387
:1033500011883046BDE8F88FA06AE76AA9EB06033A
:103360003F1A9F4228BF1F46402F1BD905F140033B
:1033700055F8042B40F8042B9D42F9D1A36A403341
:10338000A3624036A26AE36A9A4204D3E169204606
:103390000439FFF795FF8BF311884E45D9D288F396
:1033A0001188CDE729463A46FDF7FCFCA36A3B4469
:1033B0003D44A3623E44E5E7026943699A4203D172
:1033C000C3681BB9184670470023FBE7836A002BCC
:1033D000F8D0043B9B1AF5D01360C368013BC3606F
:1033E000C3691A44836902619A4224BF436A036134
:1033F000002383620123E5E700F034B9034B002288
:1034000058631A610222DA60704700BF000C004066
:10341000014B0022DA607047000C0040014B5863FA
:10342000704700BF000C0040FEE7000010B5174CCD
:10343000FEF7ECFCFEF70EFE802215492046FEF753
:1034400093FD012344F8180C0374124B124AD968F7
:1034500021F4E0610904090C0A431049DA60CA68E2
:1034600042F08072CA600E490A6842F001020A60A6
:103470001022DA77202283F82220002383F3118898
:1034800062B60848BDE81040FEF790BDAC2A0020A7
:10349000983C000800ED00E00003FA05F0ED00E0C4
:1034A000001000E0A03C00082DE9F84F1F4CDFF8A9
:1034B0008090656904F114074FF00008D9F82430B2
:1034C000266AAA689E1B96421DD34FF0200AAA685E
:1034D000236AD5F80CB0134423622B68BB425F60AB
:1034E000A6EB02066361C5F80C8001D1FFF790FFDF
:1034F00088F311882869D8478AF311886569AB6811
:103500009E42E4D2DAE76269BA420CD09168236243
:103510008E1B9660A86802282CBF1818981CBDE85E
:10352000F84FFFF77BBFBDE8F88F00BF842A00206B
:10353000000C0040034B59685A68521A9042FBD85D
:10354000704700BF001000E04B6843608B688360E9
:10355000CB68C3600B6943614B6903628B6943624B
:103560000B6803607047000008B5224B22481A69B7
:1035700040F2FF110A431A611A6922F4FF7222F025
:1035800001021A611A691A6B0A431A631A6D0A4317
:103590001A651A4A1B6D1146FFF7D6FF184802F14B
:1035A0001C01FFF7D1FF174802F13801FFF7CCFFEC
:1035B000154802F15401FFF7C7FF144802F17001EA
:1035C000FFF7C2FF124802F18C01FFF7BDFF11485F
:1035D00002F1A801FFF7B8FF0F4802F1C401FFF79D
:1035E000B3FF0E4802F1E001FFF7AEFFBDE808406F
:1035F00000F0A4B80038024000000240C03C0008BF
:103600000004024000080240000C0240001002408A
:103610000014024000180240001C0240002002403A
:1036200008B500F0FBF9FFF701FFFFF739F8BDE837
:103630000840FEF719BE000070470000084B1A69E9
:10364000920710B508D500241C61202383F311884C
:10365000FFF72AFF84F31188BDE81040FFF742B856
:10366000000C0040104B1A6C42F008021A641A6EEB
:1036700042F008021A660D4A1B6E936843F0080375
:1036800093600B4B53229A624FF0FF32DA620022B2
:103690009A615A63DA605A6001225A6108211A60FD
:1036A0003220FDF77DBD00BF00380240002004E05D
:1036B000000C00401F4B1A696FEAC2526FEAD252E7
:1036C0001A611A69C2F308021A614FF0FF301A69D1
:1036D0005A69586100215A6959615A691A6A62F037
:1036E00080521A621A6A02F080521A621A6A5A6A80
:1036F00058625A6A59625A6A1A6C42F080521A64C5
:103700001A6E42F080521A661A6E0B4A106840F424
:1037100080701060186F00F44070B0F5007F1EBF1D
:103720004FF4803018671967536823F400735360AF
:1037300000F054B90038024000700040304B4FF0A8
:1037400080521A642F4A4FF4404111601A6842F0C7
:1037500001021A601A689207FCD59A6822F00302E7
:103760009A60274B19469A6812F00C02FBD1186830
:1037700000F0F90018609A601A6842F480321A600A
:103780000B689B03FCD54B6F43F001034B671C4B4D
:103790005A6F9007FCD51C4A5A601A6842F0807232
:1037A0001A60184A53685904FCD5154B1A689201DF
:1037B000FCD5164A9A60164B1A68164B9A42164B5D
:1037C0001BD1164A1168164A914216D140F20512D1
:1037D0001A600B4B9A6842F002029A609A6802F0F3
:1037E0000C02082AFAD15A6C42F480425A645A6E8A
:1037F00042F480425A665B6E704740F20572E7E71A
:103800000038024000700040085440070094883897
:10381000002004E011640020003C024000ED00E0C4
:1038200041C20F41084A08B5536911680B4003F0C3
:103830000103536123B1054A13680BB150689847DF
:10384000BDE80840FEF74EBF003C01409C2500202B
:10385000084A08B5536911680B4003F0020353612D
:1038600023B1054A93680BB1D0689847BDE808407A
:10387000FEF738BF003C01409C250020084A08B5EF
:10388000536911680B4003F00403536123B1054AE7
:1038900013690BB150699847BDE80840FEF722BF95
:1038A000003C01409C250020084A08B55369116876
:1038B0000B4003F00803536123B1054A93690BB130
:1038C000D0699847BDE80840FEF70CBF003C0140B6
:1038D0009C250020084A08B5536911680B4003F085
:1038E0001003536123B1054A136A0BB1506A98471C
:1038F000BDE80840FEF7F6BE003C01409C250020D4
:10390000174B10B55C691A68144004F478725A6158
:10391000A30604D5134A936A0BB1D06A9847600690
:1039200004D5104A136B0BB1506B9847210604D590
:103930000C4A936B0BB1D06B9847E20504D5094A4A
:10394000136C0BB1506C9847A30504D5054A936CD2
:103950000BB1D06C9847BDE81040FEF7C3BE00BF66
:10396000003C01409C2500201A4B10B55C691A6888
:10397000144004F47C425A61620504D5164A136D62
:103980000BB1506D9847230504D5134A936D0BB1C5
:10399000D06D9847E00404D50F4A136E0BB1506EFA
:1039A0009847A10404D50C4A936E0BB1D06E98478A
:1039B000620404D5084A136F0BB1506F9847230473
:1039C00004D5054A936F0BB1D06F9847BDE81040FE
:1039D000FEF788BE003C01409C250020062108B56A
:1039E0000846FDF7DDFB06210720FDF7D9FB062180
:1039F0000820FDF7D5FB06210920FDF7D1FB0621A4
:103A00000A20FDF7CDFB06211720FDF7C9FB062193
:103A10002820BDE80840FDF7C3BB000008B5FFF74C
:103A200049FEFDF7A7FAFDF761FDFDF74DFFFDF734
:103A300021FEFFF701FEBDE80840FFF7DDBC0000F6
:103A4000034611F8012B03F8012B002AF9D1704726
:103A5000121012131211000053544D3332463F3FDF
:103A60003F00000000000000583A00083F0000003E
:103A7000130400009C3A00083F00000019040000F5
:103A8000A63A00083F00000021040000B03A0008F8
:103A90003F000000C42A00201C26002053544D3350
:103AA00032463430780053544D3332463432780045
:103AB00053544D3332463434365858000096000083
:103AC00000000000000000000000000000000000F6
:103AD00000000000B5140008A1140008DD1400085F
:103AE000C9140008D5140008C1140008AD1400085A
:103AF00099140008E914000800000000ED15000802
:103B0000D915000815160008011600080D16000842
:103B1000F9150008E5150008D11500087116000810
:103B20000000000001000000000000000200000092
:103B3000000000001918000881180008400040002B
:103B40005C2F00206C2F002002000000000000000D
:103B50000300000000000000C5180008000000007D
:103B6000100000007C2F0020000000000100000079
:103B70000000000020320020010102004172647543
:103B800050696C6F740025424F415244252D424CC0
:103B9000002553455249414C2500000009220008E8
:103BA0007121000885170008ED210008430000007E
:103BB000B43B000809024300020100C032090400BE
:103BC000000102020100052400100105240100018A
:103BD000042402020524060001070582030800FFF1
:103BE00009040100020A000000070501024000006C
:103BF000070581024000000012000000003C0008A0
:103C00001201100102000040091241570002010296
:103C1000030100000403090425424F4152442500DA
:103C20004634425900303132333435363738394131
:103C300042434445460000000040000000400000B0
:103C400000400000004000000000010000000200F1
:103C5000000002000000020000000200000002005C
:103C60000000020000000200000000000D1A000821
:103C7000ED1C0008991D0008400040008032002023
:103C800080320020010000009032002080000000FF
:103C900040010000030000006D61696E000000003B
:103CA000B83C000898320020903400200100000049
:103CB000293400080000000069646C650000000001
:103CC0000001802A00000000AAAAAAAA00010000A0
:103CD000FFFF00000000000000A00A00000000013B
:103CE00000000000AAAAAAA800000001FFFF00002F
:103CF00000000000000000000000000000000000C4
:103D0000AAAAAAAA00000000FFFF0000000000000D
:103D1000000000000028000000000000AAAAAAAAD3
:103D200000140000FFFF000000007007000000000A
:103D30005000004000000000AAAAAAAA000000400B
:103D4000FFFF000000000000000000000000000075
:103D500000000000AAAAAAAA00000000FFFF0000BD
:103D60000000000000000000000000000000000053
:103D7000AAAAAAAA00000000FFFF0000000000009D
:103D80000000000000000000000000000A00000029
:103D90000000000003000000000000000000000020
:103DA0000000000000000000000000000000000013
:103DB0000000000000000000000000000000000003
:103DC000FF0096000000000804000000143C0008FA
:103DD00000000000000000000000000000000000E3
:083DE0000000000000000000DB
:00000001FF
